:1000000019C034C033C0B7C431C030C02FC02EC0F7
:100010002DC02CC02BC0F2C5E6C628C027C026C004
:1000200025C02FC7FAC6F9C6F8C6FAC6FCC601C76E
:100030000CC721C711241FBE20E0A89521BD20E0D8
:1000400025BFE0E1FFE0A0E6B0E020E003C0C895F6
:1000500031960D92A236B207D1F7A2E6B0E020E0C9
:1000600001C01D92A63FB207E1F7ABC100C01895D1
:1000700088231CF0681730F404C060956F5F861702
:1000800008F4862F9927089587B9369A86B184FF98
:10009000FDCF0FB6F89484B10FBE95B1089587B91E
:1000A000369A86B184FFFDCF0FB6F89484B10FBEA7
:1000B00095B1969587959695879599270895282FB8
:1000C00030E0E0E0F0E845E050E8222314F46E2749
:1000D0007F27220F972F862F80709078892B41F0F1
:1000E000660F771F642775273F5F383070F303C0B2
:1000F000660F771FF9CF972F862F0895CF93DF9341
:10010000D091AE00DE5F1092800010927F00C0E0C0
:10011000CD1788F4EC2FFF27E355FF4F60917F0048
:10012000709180008081CBDF9093800080937F006E
:10013000CF5FCD1778F32DEA30E0F32FE22FEC0FED
:10014000F11D80917F0090918000892F99278083F5
:10015000CF5FF32FE22FEC0FF11D80917F008083A2
:10016000DF91CF910895CF93DF93D0919400DC5F1E
:1001700060E070E0C0E0CD1758F4EC2FFF27ED569B
:10018000FF4F80819CDF682F792FCF5FCD17A8F3B9
:10019000972F862FDF91CF910895982F963628F4C8
:1001A00086958695890F99270CC09A3940F09095CD
:1001B0009F5F892F86958695980F90959F5F892FD1
:1001C00099270895882341F0662319F0681718F4D9
:1001D000861B992703C0681B862F99270895CF9304
:1001E000DF93D82FC62FDC17F9F0DD23D9F06C2F61
:1001F0008D2FE8DF282F822F9927982F88270197A6
:10020000CD1770F42D2F222341F03327732F622F47
:1002100056D6972F862F992709C08FEF90E006C0FA
:100220002C2FF1CFCC2319F780E090E0DF91CF9114
:10023000089582E034DF80937600843640F5F894A8
:1002400090E0969A9F5F9832E0F382E087B9369A01
:10025000AE9A90E0F8949F5F9630E0F3AE9896984F
:10026000789486B184FFFDCF0FB6F89484B10FBEA9
:1002700095B196958795969587958093F000909186
:100280007600981708F041C0891B8093F00082E047
:1002900006DF80937600843640F5F89482E087B9D3
:1002A00090E0959A9F5F9832E0F3369A90E0F89448
:1002B0009F5F9630E0F39598789486B184FFFDCFE8
:1002C0000FB6F89484B10FBE95B196958795969523
:1002D000879580936C00959880916C009091760042
:1002E000981780F4891B80936C0080917900882393
:1002F00079F090916C008091F00080936C00909365
:10030000F00006C010926C00F0CF1092F000BFCF4A
:10031000089590E0AA9AAC9AAB9A2091F000283008
:1003200020F480916C008830A0F060916C00822FE6
:1003300056DF893760F09091F00080916C0089174A
:1003400018F491E0AA9805C093E0AC9802C092E03E
:10035000AB98892F992787FD90950895813059F1A1
:1003600083B380FF03C083B381FF1BC09091620001
:1003700083B380FF0BC0923329F0992309F5909342
:1003800079001EC081E080937900F7CF83B381FFAD
:10039000F2CF992381F3892F815080936200982FA7
:1003A000EACF90916200923318F7892F8F5F809384
:1003B0006200982FDDCF1092620010927900D0CFAA
:1003C0000895CFE5D2E0DEBFCDBF82E083BF8FE9E5
:1003D00082BB8FEF81BB18BA8FE187BB1ABA1BBAF9
:1003E00085E886B98FE185BB8CEF84BB8BE085BD4A
:1003F00088E183BD80E809B6082A09BE8FE289B981
:10040000549A579A1092F5001092E60010927900D3
:10041000FF24F092CE0082E38093A70084E68093CD
:10042000750010926F0010926E001092ED00109205
:10043000EC00F0928400F092AA00F092F400F092A6
:100440008F00F0926D00F0927700F092E800F09249
:100450006B00949A81E082DF1092E700979878947D
:100460008091840080FFB9C1979880916B008823A8
:10047000B9F38CE00FB6F894A89581BD0FBE97989C
:1004800080E06CDF80E00BDE8093EB0083E007DE32
:100490008093EF0086E003DE8093780087E0FFDD45
:1004A0008093AC008091EF00813608F094C192985F
:1004B0008091AA00882309F48CC180916B00882365
:1004C00009F485C18091AC00893408F47EC1939809
:1004D000C091D600C695C695C052D091D700D6958A
:1004E000D695D0528091E600C81B8091F500D81BAC
:1004F0006FE18C2FBDDDC82F6FE18D2FB9DDD82FB7
:100500006C2F772767FD7095262F372F77230CF4F4
:1005100057C1932F822F880F991F820F931F24E6B4
:1005200030E0732F622F681B790B8D2F992787FD81
:100530009095B3D4732F622FC2D4972F862FD82FC4
:100540008C2F8D1B6FE194DD8093F400CD0F6FE154
:100550008C2F8EDD80938F008091F4008D3F08F406
:100560002AC11092F40090918F009D3F08F41DC1A4
:1005700010928F0090E0992331F099230CF413C16D
:10058000945090938F008091F400882331F0882359
:100590000CF407C184508093F4008091F400FDDDD9
:1005A0008093F40080918F00F8DD80938F0080911C
:1005B0006B00882309F4F2C08091DA0080936D000B
:1005C0008091DB00809377008091770083FF0EC0DD
:1005D0008091D6008695869580528093E600809122
:1005E000D7008695869580528093F50010EEC0E284
:1005F00009EF97E080916D0083FF1DC0C093F40068
:10060000C0938F0085B382FFC6C085B384FFBEC090
:1006100085B383FFB6C08091F4008D1B6FE128DDA8
:100620008093F40080918F008D0F6FE121DD809326
:100630008F0080916D0086FF11C01093F400C0936D
:100640008F0085B382FF98C085B384FF90C085B3C7
:10065000982F987083FF86C080916D0080FF0FC037
:10066000C093F40010938F0085B385B384FF75C0E9
:1006700085B3982F987083FF6BC080916D0085FFC4
:100680001BC01093F40010938F0085B382FF5DC0F0
:1006900085B384FF55C085B383FF4DC08091F400BE
:1006A0008D1B6FE1E5DC8093F40080918F008D0F4E
:1006B0006FE1DEDC80938F0080917D008823B1F1B3
:1006C00028DEDAD080916D0081FF28C080918D00F6
:1006D00081FF1DC0909179009923B9F027E18091A5
:1006E0007700882344F486E98093A70090917900ED
:1006F000992349F027E09F1509F471C0F92E86E986
:100700008093A7006CC027E1F6CF27E0E8CF80E216
:1007100091E090936F0080936E00DCCF80918D000C
:1007200081FFD8CF8BE480937500D4CF80E680938F
:100730007D007FDDC5CF1093F40010938F00AECF06
:100740001093F40000938F00A6CF0093F400A0CF85
:100750009093F40090938F0090CF1093F400C09387
:100760008F0086CF9093F40090938F0075CF1093F5
:10077000F400C0938F006BCF10938F00C093F400F0
:1007800063CFC093F400C0938F0045CF9093F400E3
:10079000C0938F003DCF90938F0037CF80936D0033
:1007A00011CF8C5FF8CE9C5FECCE892F81508430C6
:1007B00008F0E1CEDDCE8150843008F0D4CED1CE29
:1007C00022273327261B370BA4CE939A81CE949AE7
:1007D00079CEC5D272CE929A6BCE979A46CE20939E
:1007E000810080916D0080938D00809177008093CF
:1007F000EE0046CEFFCF982F992349F035EA21E04D
:1008000032BF28BF88B780FFFDCF9150C9F7089548
:10081000CF93C82FCC2321F084E6EDDFC150E1F760
:10082000CF9108958058681708F5982F961B9695D4
:100830009695D1F020E02917E0F4681738F44F5F5F
:100840005F4F4038510514F04FE750E0861740F4F1
:10085000415050403FEF4038530714F440E85FEFF9
:100860002F5F291750F305C091E0E4CF962F981B16
:10087000DECF952F842F08958091F4008EDC809335
:10088000F40080918F0089DC80938F008091F400C8
:1008900084DC8093F40080918F007FDC982F90930C
:1008A0008F0080917900882351F08091F400809529
:1008B0008F5F80938F0090959F5F9093F40090914D
:1008C000F400992309F447C08AE08093F10099234A
:1008D00089F184E0E4DB8093D20085E0E0DB809363
:1008E000820040916300509164006091D200809139
:1008F0008F0098DF909364008093630040916500BF
:1009000050916600609182008091F4008BDF282F67
:10091000392F309366002093650080916300909199
:100920006400909391008093900030937200209324
:10093000710017C080918F00882359F68091F100D3
:10094000882339F6109264001092630010926600BA
:100950001092650006C080918F00882309F0B4CF03
:10096000B6CF0895992324F080958F77992702C0F8
:100970008F77907008951F920F920FB60F921124E7
:100980002F933F934F935F936F937F938F939F9397
:10099000AF93BF93EF93FF9380917D00882319F06D
:1009A000815080937D0080916E0090916F00892B23
:1009B00049F080916E0090916F00019790936F00C5
:1009C00080936E0080918500882309F404C1AD9A5C
:1009D00080918500815080938500809168008150CE
:1009E00080936800882309F4BBC080917C00882331
:1009F00009F4A6C080916A00882309F494C080910C
:100A00007A0088BB10927A009091F200963038F408
:100A100080917400813009F082E080937A00892F00
:100A200081508093F2008F3F09F468C09091690073
:100A3000963050F48091D000813009F45BC08091F1
:100A40007A00886080937A00892F815080936900B2
:100A50008F3FD9F1809178008F3108F0AE988531C1
:100A600008F4AE9A823310F010927A008091F4006C
:100A7000882301F18091E7008130C9F080916B00FB
:100A8000882391F080916E0090916F00892B09F47A
:100A9000A4C080917500882309F09FC080917A00DE
:100AA000806180937A0099C080937A00EBCF109296
:100AB0007A00E4CF80918F008823E1F68091F100E5
:100AC0008823C1F680937A00D5CF809171009091F0
:100AD000720048DF8B5F8093690080917100909174
:100AE0007200992324F081E08093D000B3CF10925C
:100AF000D000B0CF80917A008460A4CF8091900024
:100B0000909191002FDF8B5F8093F2008091900095
:100B100090919100992324F081E08093740086CF16
:100B20001092740083CF8CE380936A008091EC0074
:100B30009091ED0001969093ED008093EC005FCFD3
:100B400084E680937C0080916A00882319F08150AC
:100B500080936A00809184008F5F809384004ACFE5
:100B600080E68093680080917C00882319F0815092
:100B700080937C0080916B00882329F080916B002A
:100B8000815080936B0080917500882329F08091BB
:100B900075008150809375008091F100882329F0C1
:100BA0008091F10081508093F1008091850088232D
:100BB00009F01BCF8091A700882351F0809181001C
:100BC000809385008091A70081508093A7000DCF6E
:100BD000809385000ACFAD9800CFFF91EF91BF9130
:100BE000AF919F918F917F916F915F914F913F91C5
:100BF0002F910F900FBE0F901F9018951F920F927C
:100C00000FB60F921124EF92FF921F932F933F93F1
:100C10004F935F936F937F938F939F93AF93BF9304
:100C2000CF93DF93EF93FF931CB1809160009927DE
:100C30008130910509F472C08230910584F4892BCA
:100C400009F071C0153509F06EC08091E9009091EE
:100C5000EA00803F910509F066C081E062C0823001
:100C6000910509F448C0039709F05DC080918C009C
:100C700063E9E62E60E0F62EFF2DEE2DE80FF11D64
:100C800010838F5F80938C00C0916700C150C09328
:100C90006700CC2309F047C066DAF92FE82F3097B8
:100CA000D1F5809193008130B1F54C2F8091940063
:100CB000282F33272E5F3F4FE217F307B4F4AE2FF0
:100CC000BF2FC3EDD0E07F2D6E2DFB2FEA2FEC0F51
:100CD000FD1FA60FB71F8C9180834F5F842F99272C
:100CE000B92FA82FA217B30784F3949885E08093B7
:100CF0006B00A89510C01093940083E0809360006F
:100D000082E080938C00812F8E5F8093670099270B
:100D10000496459744F01092600005C0109393002C
:100D200082E080936000812F99279093EA0080935E
:100D3000E900FF91EF91DF91CF91BF91AF919F912A
:100D40008F917F916F915F914F913F912F911F9163
:100D5000FF90EF900F900FBE0F901F9018951F936C
:100D600081E08093AD0012E08093AF008091F400A9
:100D70008093B00080918F008093B10080917800C3
:100D80008093B2008091EF008093B3008091AC001B
:100D90008093B40080918A008093B5008091AB006D
:100DA0008093B60080916D008093B70080917700AA
:100DB0008093B800809184008093B900912F955F53
:100DC000809182008093BA008091D2008093BB0012
:100DD0009093AE0093D91093AA00539A559A8FEF2F
:100DE0008CB91F9108951F920F920FB60F92112484
:100DF0002F938F939F93AF93BF93EF93FF93209184
:100E0000AA00822F9927AA27BB27F92FE82FE930BC
:100E1000F105B8F5EF5EFF4F09948FEF8CB905C06F
:100E200080EF8CB902C085E58CB92F5F2093AA00B2
:100E300028C0109273008091AE008C5F8093E50013
:100E40008091AA008F5F8093AA0090917300EDEAD1
:100E5000F0E0E90FF11D80818CB99F5F90937300E2
:100E60008091E50081508093E500882351F488E06B
:100E70008093AA0006C01092AA008FEF8CB95598F3
:100E80005398FF91EF91BF91AF919F918F912F91C7
:100E90000F900FBE0F901F9018955527002480FFCC
:100EA00002C0060E571F660F771F6115710521F0EE
:100EB00096958795009799F7952F802D089597FB24
:100EC000092E07260AD077FD04D00CD006D00020CA
:100ED0001AF4709561957F4F0895F6F79095819576
:100EE0009F4F0895AA1BBB1B51E107C0AA1FBB1F40
:100EF000A617B70710F0A61BB70B881F991F5A95A6
:100F0000A9F780959095682F792F8A2F9B2F0895A8
:020F10000000DF
:00000001FF
